:100000000C9418010C9435010C9435010C943501B5
:100010000C9435010C9435010C9435010C94350188
:100020000C9435010C9435010C94991B0C946B1CA9
:100030000C94A0160C9435010C9435010C943501E8
:100040000C9435010C9435010C9435010C94350158
:100050000C9435010C9428170C9435010C9435013F
:100060000C9435010C9435010C9435010C94350138
:100070000C9435010C9435010C9435010C94350128
:100080000C9435010C9435010C9435010C94350118
:100090000C9435010C9435010C9435010C94350108
:1000A0000C9435010C9435010C9435015D035D030E
:1000B00089038903F1030F04270527051A04B304F4
:1000C000C404C404D81CFF1CF71DFF1CF71D4B1DE6
:1000D0006E1DF71DC51DD41D00001A00000018007C
:1000E0000C00120013000400160007000B000D00A6
:1000F0000E000F00120346006900670068007400DC
:1001000050006100640000001A0341006C006900A7
:100110007300470072006100760065004E006900C0
:100120006C0000000403090409023B00020100A066
:10013000FA09040000010301010009211101000175
:1001400022400007058103080001090401000103A2
:10015000000000092111010001227B000705820334
:10016000200001120100020000000867771C48010E
:10017000000102000105010902A10185020901A196
:100180000005091901290815002501950875018147
:10019000020501093009311581257F950275088115
:1001A0000609381581257F950175088106050C0A19
:1001B00038021581257F950175088106C0C00501AB
:1001C0000980A101850319012AB700150126B7008E
:1001D000950175108100C0050C0901A10185041964
:1001E000012AA002150126A002950175108100C008
:1001F00005010906A101050719E029E715002501F8
:10020000950875018102950175088101050719009E
:1002100029FF150026FF00950675088100050819BD
:10022000012905950575019102950175039101C09C
:1002300011241FBECFEFDAE0DEBFCDBF11E0A0E09A
:10024000B1E0E4E5FDE302C005900D92A438B107EA
:10025000D9F722E0A4E8B1E001C01D92A133B207B2
:10026000E1F70E94E8100C94A81E0C94000081E0B5
:10027000089581E008950C94390108950C943D018E
:100280001F93CF93DF9300D000D01F92CDB7DEB77E
:1002900049835A836B833091870189819A81311117
:1002A00014C0662359F0222349F00E946407182FD6
:1002B000682F89819A810E940D0703C00E94380728
:1002C000182F69817A81812F04C00E946407698197
:1002D0007A810F900F900F900F900F90DF91CF9138
:1002E0001F910C94850EFC01262F40815181628163
:1002F000738184810C94400181E00895CF93DF9352
:10030000EC0160E00E947301BE01DF91CF910C947B
:100310003E010C94CB0F0C94C70F08950E94B705B3
:100320000E948D012FEF84E39CE02150804090409B
:10033000E1F700C000000C944E170F931F93CF936A
:10034000DF938C0161E00E947301EC01B8010E940F
:100350003B018823F1F1B801CE010E946A15882380
:10036000C1F1B801CE010E947E13882391F1B8013A
:10037000CE010E94C614882361F1F801828188238E
:1003800009F1CB358DE5D807C1F050F4C115FCE576
:10039000DF0781F0CF3DDC45A9F40E949B0C19C01A
:1003A000CC35EDE5DE0761F0CD35DD4559F40E9431
:1003B000DE0B08C00E948E010CC00E94E70B02C039
:1003C0000E94EA0BC801DF91CF911F910F910C940D
:1003D000370180E0DF91CF911F910F9108950E9426
:1003E00081160C9408020E940B020C948716089543
:1003F0000C94F70181E008950C94FA010895CF93CD
:10040000C82F0E94F8018C2F0E94FC01CF91089503
:1004100080E00C94FF010E94C6150C94FF010E941D
:10042000C61590918601891721F0809386010C945E
:10043000FF010895CF93DF93CDB7DEB72B970FB6AB
:10044000F894DEBF0FBECDBF4F83588769877A8788
:100450008B8761110E942A0B9E012F5F3F4F86E020
:10046000F90111928A95E9F785E0FE013796D901E5
:1004700001900D928A95E1F789819A814C815D8185
:10048000452B31F09F3F31F491E08F3F19F403C0C9
:1004900091E001C090E090FF09C049815A816B81D1
:1004A0007C818D819E810E944B0A05C0C9010E94FA
:1004B0007C018111F2CF2B960FB6F894DEBF0FBEF0
:1004C000CDBFDF91CF910895FC01808191810E9481
:1004D000A6070895CF93882309F450C0C82F8CEF46
:1004E0008C0F813AD0F46C2F80910201909103011E
:1004F0000E942316882349F06C2F8091020190916D
:1005000003010E945B160E944C0B6C2F809102012C
:10051000909103010E9459160CC080E28C0F883024
:1005200058F4C77081E001C0880FCA95EAF70E94AD
:100530000D0BCF910C944C0BEBE5EC0FE33040F43A
:10054000F0E0E95BFE4F808190E0CF910C94EB15D9
:10055000E8E5EC0FE73150F4F0E0EE0FFF1FE75E47
:10056000FE4F80819181CF910C940116CD3E30F0E9
:100570008C2F0E946D11CF910C943F12CF91089552
:10058000882389F19CEF980F913A40F4682F80916D
:100590000201909103010E945B160DC090E2980F3A
:1005A000983058F4877091E001C0990F8A95EAF766
:1005B000892F0E94130B0C944C0B9BE5980F9330E2
:1005C00020F480E090E00C94EB1598E5980F9731BB
:1005D00020F480E090E00C9401168D3E20F00E9403
:1005E000C8110C943F1208951F93CF93DF93182FD7
:1005F000EB010E946A02209741F08FE99FE001978A
:10060000F1F700C000002197F6CF812FDF91CF9145
:100610001F910C94C002893319F060E070E002C0B1
:1006200060E570E00C94F402882321F00E940D0B29
:100630000C944C0B0895882321F00E94130B0C940A
:100640004C0B0895CF92DF92EF92FF920F931F937E
:10065000CF93DF937C01D62FC72FFC011281058138
:1006600002950F700E94030B8823B9F01123A9F0A3
:100670008C2F807F803421F080E28D0F883068F0ED
:1006800080911B0282FD09C082E00E94AC0B0E9497
:10069000030B91E0D82ED92601C0D12CCC2EC294C8
:1006A0008FE0C8228C2D90E08C30910508F0CFC1EE
:1006B000FC01EA5AFF4F0C943F1E8C2F807FCF70B5
:1006C000882311F0C295C07F112399F0CC2309F43F
:1006D000AAC180E28D0F883010F0D11104C08C2F98
:1006E0000E940D0B03C08C2F0E941D0B0E944C0B0F
:1006F0009AC18D2F0E94C002CC2309F4A8C180E2C8
:100700008D0F883038F1DD2329F18C2F0E94230BC7
:1007100024C08C2F807FCF70803211F0C295C07FB3
:10072000DD2319F0D130A1F13DC080911B0282FF81
:1007300017C0112349F0CC2329F08C2F0E940D0BF8
:100740000E944C0B80E070C180E00E94C002CC236C
:1007500009F47DC18C2F0E94130B0E944C0B77C1B2
:10076000112371F0002341F0013031F40E942D0B70
:100770008C2B0E94350B6BC10E942D0B8C2B1DC046
:10078000002319F0013009F462C10E94420B25C018
:10079000112321F0063008F05AC10EC0053008F0D0
:1007A00056C11BC0112361F0002331F0F701858190
:1007B00080FF39C18F7085838C2F0E94140347C13D
:1007C000002359F0D93309F03FC1FFEF07EE13E0E2
:1007D000F15000401040E1F735C18C2F0E941B03FF
:1007E00036C18C2F86958695837019F0813061F023
:1007F0002EC1112321F08D2F9C2F937002C080E019
:1008000090E00E94EB152BC1112321F08D2F9C2F1E
:10081000937002C080E090E00E94011620C18D2FED
:10082000112319F00E946D1102C00E94C8110E948C
:100830003F1215C18C2F837009F047C011110BC1F5
:100840002D2F229526952770220F220F6D2F6F7066
:10085000862F90E0A0E0B0E0022E04C0880F991F20
:10086000AA1FBB1F0A94D2F7D4FF10C04FE050E07C
:1008700060E070E004C0440F551F661F771F2A9583
:10088000D2F7409550956095709503C040E050E0D8
:10089000BA01C695C695C3708A019B01082B192B16
:1008A0002A2B3B2BC901B801C23049F058F4C130A2
:1008B00019F00E942306CFC00E941106CCC00E94EE
:1008C0003506C9C00E940F06C6C0112319F08C2F2F
:1008D000817001C08695882309F4BDC02D2F229513
:1008E00026952770220F220F6D2F6F70862F90E0B4
:1008F000A0E0B0E0022E04C0880F991FAA1FBB1F02
:100900000A94D2F7D4FF10C04FE050E060E070E0EE
:1009100004C0440F551F661F771F2A95D2F74095D4
:1009200050956095709503C040E050E0BA01C695BF
:10093000C695C3708A019B01082B192B2A2B3B2BD0
:10094000C901B801C23049F058F4C13019F00E9411
:10095000E80681C00E94D6067EC00E94FA067BC0CF
:100960000E94490678C0CF70112339F08C2F0E9465
:100970006F068D2F0E9414036EC08D2F0E941B03E3
:100980008C2F0E94900667C0D23F21F128F4D03FFF
:1009900041F0D13FC1F043C0D33F19F1D43F79F0CA
:1009A0003EC0112341F0053008F051C08C2F8F71EB
:1009B0000E94B5064CC0063008F049C0F7CF8091C0
:1009C0001B0282FF18C0112339F08C2F8F710E94F7
:1009D0006F063DC01123C9F38C2F8F710E949006C2
:1009E00036C0112329F08C2F8F710E945A062FC018
:1009F0000E9455062CC0112349F0CF718C2F0E9404
:100A00006F0663E08C2F0E94910B21C081E00E9451
:100A1000AC0B0230E0F082E00E94AC0B18C0112356
:100A200031F0002391F28D2F0E946A0210C0002342
:100A300099F2D93349F41FEF27EE33E011502040EB
:100A40003040E1F700C000008D2F0E94C00288EF07
:100A50008C0D843020F40E94C6150E94FF01DD2019
:100A6000C9F00E94FF0A80FD15C0F70112820E94A2
:100A7000F90A0E946F06C7010E946B050E94F90ADD
:100A8000DF91CF911F910F91FF90EF90DF90CF906A
:100A90000C949006DF91CF911F910F91FF90EF90F2
:100AA000DF90CF9008950F931F93CF93DF93EC01C6
:100AB000688179818A810E94B1078C010E940C07AC
:100AC0000E94FD05B801CE010E942203DF91CF9163
:100AD0001F910F910895CF93DF93EC019881898145
:100AE0002B813C81232B31F08F3F31F481E09F3FFC
:100AF00019F403C081E001C080E080FD1DC0CE017B
:100B00000E949D01811110C00E94030B8823A1F057
:100B10008A81882389F080911B0282FD0DC082E0CA
:100B2000DF91CF910C94AC0BCE010E945305CE0106
:100B3000DF91CF910C947E01DF91CF91089580E0F9
:100B400090E00E94EB1580E090E00E9401160E9468
:100B50002A0B0E944C0B0E9470130C943F12809140
:100B60000201909103010E945D160C949F050E9462
:100B70001A0B0C94AF0592959F70963079F010F493
:100B8000925001C09A50923068F4803F69F018F496
:100B9000883E40F409C0843F29F406C0883E20F016
:100BA000813F11F080E0089581E00895FC0180818B
:100BB00091810E94A6070E94BB050895CF93DF9301
:100BC00000D000D01F92CDB7DEB70F900F900F90DE
:100BD0000F900F90DF91CF910895CF93DF9300D0C6
:100BE00000D000D0CDB7DEB726960FB6F894DEBFA2
:100BF0000FBECDBFDF91CF910895089508950C9455
:100C0000FE050C94FF050E94010660939601709307
:100C1000970180939801909399010C949F050C94EF
:100C200003060F931F930091960110919701209155
:100C3000980130919901602B712B822B932B1F917E
:100C40000F910C9403060F931F930091960110913E
:100C5000970120919801309199016023712382239B
:100C600093231F910F910C9403060F931F930091F0
:100C70009601109197012091980130919901602778
:100C80007127822793271F910F910C9403060C94D0
:100C9000FE050E9447066093920170939301809332
:100CA0009401909395010C949F0560E070E0CB0156
:100CB0000C9449060F931F9341E050E060E070E010
:100CC0008A019B0104C0000F111F221F331F8A9548
:100CD000D2F7C901B8011F910F910C9449060F93E7
:100CE0001F9341E050E060E070E004C0440F551FE6
:100CF000661F771F8A95D2F7809192019091930198
:100D0000A0919401B09195018A019B01082B192BA8
:100D10002A2B3B2BC901B8011F910F910C94490656
:100D20000F931F9341E050E060E070E004C0440F77
:100D3000551F661F771F8A95D2F74095509560958D
:100D400070958091920190919301A0919401B0913E
:100D500095018A019B01082319232A233B23C901FA
:100D6000B8011F910F910C9449060F931F9341E016
:100D700050E060E070E004C0440F551F661F771F0D
:100D80008A95D2F78091920190919301A09194015C
:100D9000B09195018A019B01082719272A273B2733
:100DA000C901B8011F910F910C9449060F931F932D
:100DB000009192011091930120919401309195013D
:100DC000602B712B822B932B1F910F910C94490652
:100DD0000F931F9300919201109193012091940120
:100DE0003091950160237123822393231F910F91EA
:100DF0000C9449060F931F93009192011091930157
:100E000020919401309195016027712782279327C3
:100E10001F910F910C944906089527E0929F800D31
:100E20001124E82FE695E695E695877051E001C01C
:100E3000550F8A95EAF785E0E89FF0011124E857FD
:100E4000FE4F20E030E070E04081CB01022E02C076
:100E5000969587950A94E2F781708195842785237A
:100E6000842781932F5F3F4F2530310569F708951F
:100E700027E0929F800D1124682F669566956695F0
:100E8000982F977085E0689FB001112440E050E0F2
:100E900080E0FB01E40FF51FE857FE4F208130E0B2
:100EA000092E02C0369527950A94E2F72170332760
:100EB000042E01C0220F0A94EAF7822B4F5F5F4F86
:100EC0004530510531F70895BF92CF92DF92EF92EE
:100ED000FF920F931F93CF93DF938C01C0909201E9
:100EE000D0909301E0909401F0909501809196014B
:100EF00090919701A0919801B0919901C82AD92A9F
:100F0000EA2AFB2ACFE1D0E0D701C6010C2E04C0AB
:100F1000B695A795979587950A94D2F780FD04C05A
:100F2000219790F7B12C07C0BC2EB8018C2F0E94DE
:100F3000980E0197A9F38B2DDF91CF911F910F91FF
:100F4000FF90EF90DF90CF90BF900895CF93DF9305
:100F5000EC010E946407BE010E94980EDF91CF91C0
:100F600008951F93CF93DF93EB019091870199230D
:100F700021F0CB010E94A60713C0882349F0CB01C2
:100F80000E946407182F682FCE010E940D0704C02D
:100F9000CB010E943807182FBE01812F0E94980EA6
:100FA000DF91CF911F9108951F93CF93DF93C0914D
:100FB0009A0116E080919B01C81799F0D0E01C9F20
:100FC000F0011D9FF00D1124E456FE4F4081518128
:100FD00062817381848195810E94ED052196C7709D
:100FE000E9CFDF91CF911F9108954091CC015091AD
:100FF000CD016091CE017091CF018091D00190918F
:10100000D1010C94ED05EF92FF920F931F93CF93B4
:10101000DF938091D10182958F7009F065C0809136
:10102000CE01882309F460C080919A01F0909B0161
:101030001091CC010091CD016091CF017091D00150
:1010400091E01F3F09F090E0C0910001D0910101B3
:10105000292F96E0E92E8F1509F446C06115710518
:1010600021F00F3F21F030E003C031E001C0322F0A
:1010700090E030FD36C0E89EF001E99EF00D1124AD
:10108000DF01A456BE4F11963C911197301329C031
:101090003C91311326C012963C911297311121C018
:1010A00013964D915C911497461B570B4C175D0797
:1010B000C0F48091D1018F7080618093D101EF5590
:1010C000FE4F80818F70806180838CEC91E00E9464
:1010D0006B05DF91CF911F910F91FF90EF900C94D2
:1010E000D40701968770B7CFDF91CF911F910F91F1
:1010F000FF90EF9008959F92AF92BF92CF92DF92B0
:10110000EF92FF920F931F93CF93DF93CDB7DEB78C
:1011100061970FB6F894DEBF0FBECDBF8C0185E09E
:10112000F801DE011D9601900D928A95E1F7D80134
:101130001296EC909091CC01E091CD012091CF01DD
:101140003091D0012115310531F0EF3F31F481E0CC
:101150009F3F19F403C081E001C080E0B82FB17057
:101160009B2E80FD47C1D8014C9111965C9111973F
:101170001396AD90BC9014978CECC82E81E0D82EBD
:10118000F090CE01B501621B730B209100013091EC
:101190000101FF2009F4D9C08091D10162177307C2
:1011A00008F095C0282F207F09F052C05E1313C0AD
:1011B000491311C0FE2CE1100EC08F708061809326
:1011C000D1010E94F507C6010E946B058091D101F3
:1011D000F80185834DC1AB2831F05F3F31F481E0E8
:1011E0004F3F19F403C081E001C080E080FD03C0DF
:1011F00081E08E2502C080E090E0F82FF170FF2E94
:1012000080FF1CC080919A0120919B0136E08217DB
:1012100009F40BC190E0389FF001399FF00D1124C3
:10122000E456FE4F6181561306C06081461303C029
:101230006281E61203C001968770E9CFFE2CEE2092
:1012400009F416C18091D10181608093D10154C00D
:101250005E1306C0491304C0E11002C0F80199C032
:10126000C8010E94D605882361F1EE2051F120913A
:10127000D101822F82958F7090E0029774F0809157
:10128000CC019091CD0198878F831986BB86AA8661
:101290002C87CE0107960E946B0586E0F801ACEC26
:1012A000B1E001900D928A95E1F70E9403080E9437
:1012B000F5070AC05E1711F1C8010E94D605811119
:1012C0002CC0C8010E946B05FF24F394D1C0282FC5
:1012D000207F81F77A2DB98AA88A6E2D89890E948C
:1012E000DE058CEC91E00E946B0586E0D6011D9234
:1012F0008A95E9F70E94F507F12CBAC04913DCCFB3
:10130000E110DACFF8018583C8010E946B0586E001
:10131000D6011D928A95E9F7ABC0EE2091F220919B
:10132000D101822F82958F7090E002970CF4B5CF97
:101330008091CC019091CD019A8389831B82BD82DB
:10134000AC822E83CE010196A6CF6217730708F0F8
:1013500044C0FE2CEE2009F4B4CF5E1330C0491314
:101360002EC02091D10120FD21C0822F82958F7047
:10137000482F50E041155105C9F0F80125834F3041
:10138000510541F08F5F982F9295907F822F8F703B
:10139000892B8583C8010E946B0586E0F801ACECBF
:1013A000B1E001900D928A95E1F73CC086E0F8012A
:1013B000ACECB1E001900D928A95E1F759C0C801FB
:1013C0000E94D605811169CF8091D10181608093FF
:1013D000D101C8010E946B054BC07A2DB98AA88A39
:1013E0006E2D89890E94DE0586E0D6011D928A95C0
:1013F000E9F718C0EE2009F464CFC8010E94D605B1
:10140000F82E882309F45DCF86E0F801ACECB1E05A
:1014100001900D928A95E1F78CEC91E00E946402B4
:101420000E9403080E94F50723C04D875E878D85C3
:101430009E850E94A607292F22952F70223028F41E
:101440009F7039F0811105C00BC0243028F49F70C3
:1014500049F4805E883020F0C8010E946B059F2C03
:10146000F92C06C0D80115969C91907F91F7F8CF82
:101470008F2D61960FB6F894DEBF0FBECDBFDF9102
:10148000CF911F910F91FF90EF90DF90CF90BF9081
:10149000AF909F9008951F93CF93DF93CDB7DEB7A2
:1014A0002C970FB6F894DEBF0FBECDBF4F83588781
:1014B00069877A878B879C87CE0107960E947B0875
:1014C0008823D1F09F8188852A853B85232B31F0A5
:1014D0008F3F31F481E09F3F19F403C081E001C0E8
:1014E00080E080FD47C04F81588569857A858B856E
:1014F0009C850E94ED053EC086E0FE013796DE0128
:10150000119601900D928A95E1F7FF81E8856A8531
:101510007B856115710531F0EF3F31F481E0FF3FCC
:1015200019F403C081E001C080E080FD23C0209158
:101530009B0130E0C90101968770992740919A017B
:1015400050E084179507F1F1F983EA837D836C837A
:1015500096E0929FD001939FB00D1124A456BE4FE8
:10156000FE01319601900D929A95E1F780939B01CF
:101570000E94D40716E080919A0190919B018917EF
:1015800071F1189FC001112484569E4F0E947B0860
:10159000882329F1E0919A011E9FF0011124E4565D
:1015A000FE4F4081518162817381848195810E94C7
:1015B000ED0580919A0190E00196877099278093BC
:1015C0009A01D9CF0E94B70510929B0110929A01FF
:1015D000ECECF1E086E0DF011D928A95E9F72C96AC
:1015E0000FB6F894DEBF0FBECDBFDF91CF911F9134
:1015F00008958091DA018595859585950895809166
:10160000DA01877008959091DA01977081E009F40A
:1016100080E008958091E50108959091E501892B7E
:101620008093E501089580959091E5018923809349
:10163000E50108951092E50108959091E401892B48
:101640008093E401089580959091E401892380932B
:10165000E40108951092E40108958091DB0108955A
:1016600008950C94300B0C94310B90911B0292FD59
:1016700008C09091DB01981721F08093DB010C9456
:10168000330B08958091DB01882329F01092DB0150
:1016900080E00C94330B0895CF93DF93E091020127
:1016A000F09103018091E5018083E0910201F091C6
:1016B000030190818091E401892B80838091DB017B
:1016C000882381F0E0910201F09103019081892B40
:1016D000808380910201909103010E94171681116D
:1016E0000E94420BC0910201D091030148E050E0FA
:1016F00062ED71E0CE010E94591E892B69F088E0ED
:10170000FE01A2EDB1E001900D928A95E1F7CE01C4
:10171000DF91CF910C94D215DF91CF9108950C9465
:10172000300B90911B0292FD10C098E0899F9001B0
:101730001124262B2093DA010E946F068091DA0192
:101740008595859585950C948F0B0C946F0610925A
:10175000DA0180E00C948F0B2091DA0180958223CE
:101760008093DA01982F977099F430E0482F082E73
:10177000000C550B2417350759F090911B0292FD70
:1017800007C08595859585950E9490060C94A70BBA
:10179000089590911B0292FB222720F9281769F0E7
:1017A00080FB92F990931B0280911A0290911B0288
:1017B0000E94170C82E00C94AC0B089580911B02E0
:1017C00082FB882780F991E089270C94C90B81E07E
:1017D0000C94C90B80E00C94C90B6FEF7FEF80E095
:1017E00090E00C94921E80E090E00E946E1E21E03A
:1017F000893E9E4F09F020E0822F089582E090E01C
:101800000C94661E83E090E00C94661ECF9384E0F7
:1018100090E00E94661EC82F82E290E00E94661E41
:101820002C2F30E0A901582BCA01CF910895CF93F6
:10183000C92F682F84E090E00E94741E6C2F82E212
:1018400090E0CF910C94741EAB01BC018FE090E04E
:101850000C94861EAB01BC0183E190E00C94861EC3
:1018600060E070E0CB010C942A0C60E070E0CB01EA
:101870000E94240C0C94300C69EE7EEF80E090E026
:101880000E94921E60E082E090E00E94741E60E080
:1018900083E090E00E94741E1092960110929701CE
:1018A000109298011092990160E084E090E00E940B
:1018B000741E60E082E290E00E94741E60E085E0A9
:1018C00090E00E94741E60E086E090E00E94741E2A
:1018D0006FEF87E090E00E94741E40E050E0BA0194
:1018E00088E090E00E94861E60E08DE090E00E941B
:1018F000741E40E050E0BA0188E190E00E94861E2C
:1019000060E087E190E00E94741E40E050E0BA0180
:101910008CE190E00E94861E60E070E080E290E042
:101920000E94921E40E050E0BA0188E190E00E94DF
:10193000861E0C94350C0C943C0C682F8EE090E0C5
:101940000C94741E0E940D176093EC017093ED01CE
:101950008093EE019093EF016093E8017093E901A9
:101960008093EA019093EB01089585B7806885BF65
:1019700085B7806885BF089581E008950C94BC0CFC
:1019800008950C94C00C0C94C00C0C94C30C0C94D3
:10199000C00C0C94C70C0C94C00C0E94B50C84E7CE
:1019A0009FE00E94BC150E94CB0C0C94C90C0E94B5
:1019B000C10C0C94C00C0E94910F0C94FE010E946B
:1019C000F8160E945E100E94DB0C0C94C50C8F92DE
:1019D0009F92AF92BF92CF92DF92EF92FF920F93BE
:1019E0001F93CF93DF93CDB7DEB72A970FB6F89446
:1019F000DEBF0FBECDBF0E946D10982E81110E94D8
:101A0000A20C86EEA82E81E0B82E00E010E0802E19
:101A1000802F0E94B50FD82EF501C1905F01C82616
:101A2000B1F40F5F1F4F0230110589F78FEF8983E3
:101A30008A831B820E9401178160782F9D838C838B
:101A400049815A816B818D810E941A022FC0809139
:101A5000F00181FD0E94BB0FE12CFF24F3948C2D3B
:101A60008F21F1F00E94BE0C882399F0EE828F82C4
:101A7000DF2081E009F480E088870E9401178160FF
:101A8000782F9A8789874E815F8168858A850E9431
:101A90001A02F801EA51FE4F8081F826F08206C052
:101AA000E394FF0CF7E0EF12DACFBBCF81E09110A7
:101AB00001C080E02A960FB6F894DEBF0FBECDBFFE
:101AC000DF91CF911F910F91FF90EF90DF90CF901A
:101AD000BF90AF909F908F9008950E94E70C0E9456
:101AE0005D120C940F02CF93DF930E949D0EEC01C8
:101AF000811521E5920708F045C0811530E593076F
:101B000008F094C0883E910528F5803E910508F0C4
:101B1000F8C0883A910570F4853A910508F07CC0C8
:101B20008130910509F475C008F4E8C0049708F005
:101B3000E8C0E4C08F3B910508F0E0C0C85AD0E08F
:101B4000CC0FDD1FC65BDE4F0990D881C02DCE01C2
:101B50009464D8C0811540E2940758F4811551E08F
:101B6000950708F0CEC08D3E910508F4C7C090657A
:101B7000C9C0C11580E4D80708F4C0C0DF70CE0129
:101B8000906AC0C0811525E59207A8F4811534E557
:101B9000930708F095C0811543E5940708F07BC0D2
:101BA000811552E5950708F061C0D82FCC27CE01EA
:101BB000816F906AA7C0C11589E5D807A0F4C11547
:101BC00028E5D20708F082C0C11536E5D30708F032
:101BD00095C08C2F0E94310F8F7190E0D82FCC27A9
:101BE000CE0190628FC0C1154AE5D40708F474C0D5
:101BF000CE0190568115904208F080C08D2F8F71D4
:101C00000E94310FDD27D0628F71AE01582BCA01BF
:101C100079C081E090E076C0C55AD0E0C858DE4F68
:101C20008881C82FD0E0CE0190646CC074E0969596
:101C300087957A95E1F7282F23703C2F337081E048
:101C400090E002C0880F991F3A95E2F79C68AC01BA
:101C5000522B9A019C2F9F709695969550E2959FD6
:101C6000E0011124C9018C2B9D2B4CC08370992756
:101C700021E030E002C0220F331F8A95E2F79C2F4B
:101C80009695969580E2989FE0011124C22BD32B64
:101C9000CE019C6837C08370992721E030E002C0F4
:101CA000220F331F8A95E2F79C2F9695969540E276
:101CB000949FE0011124C22BD32BCE019A6822C03D
:101CC000D82FCC27CE01846F906A1CC0DC2FCC2784
:101CD000CE01806F906A16C08C2F8F700E94310FDA
:101CE00094E0D695C7959A95E1F7CF70D0E0DC2FB8
:101CF000CC27D0699E01282BC90104C080E090E068
:101D000001C0CE01DF91CF9108952EE0829FC001E6
:101D10001124FC0127E0729FE00DF11D1124E60F54
:101D2000F11DEE0FFF1FE852FF4F8591949108952A
:101D30000E94850E0E94730D08958238910569F105
:101D4000B0F48133910509F46DC048F489329105EE
:101D500009F463C08A32910509F469C00895853396
:101D6000910509F455C089339105B9F00895833E72
:101D7000910569F138F4803E9105B1F0823E9105FC
:101D800009F10895863E9105A9F1873E9105B9F1C3
:101D9000843E910509F064C023C020911A0220FD01
:101DA0004FC021FD4DC0089580911A0280FD44C0AE
:101DB00080911B0280FF44C080911A0284FD42C0C2
:101DC00083EE4DC080911A0282FF38C0F5CF80911A
:101DD0001A0282FD33C080911B0280FD31C0ECCF1E
:101DE00080911B0281FF32C080911A0284FD2AC0BB
:101DF00087EE35C080911A0283FF26C0F5CF80910F
:101E00001A0283FD21C080911B0281FD1FC0ECCF0F
:101E100080911A0285FD1CC01DC080911A0285FDAB
:101E200019C016C080911A0286FD16C017C0809195
:101E30001A0286FD13C010C089E311C082EE0FC0E4
:101E400080EE0DC080E00BC086EE09C084EE07C0B6
:101E500089E205C085E303C08AE201C081E390E026
:101E6000089590911A0292FF0DC0282F28712830F2
:101E700019F4877F846006C0282F2471243011F460
:101E80008B7F886093FF0DC0282F2871283119F4AB
:101E9000877E846106C0282F2471243111F48B7E43
:101EA000886120911B0220FF0DC0382F3871383017
:101EB00019F4877F816006C0382F3171313011F4F9
:101EC0008E7F886021FF0DC0282F2871283119F4DA
:101ED000877E816106C0282F2171213111F48E7E09
:101EE000886194FD877E089580E008950C94ED0B41
:101EF0000E946D102FEF86E791E0215080409040C6
:101F0000E1F700C000000E946D1080E00E94B50F54
:101F100080FF04C00E94760F0C944E1708950C9415
:101F2000780F0E94F30B811102C00E949B0C0E944B
:101F3000FE0B8093F0010E94060C90931B0280938D
:101F40001A020E948F0F0E94020C682F70E080E03E
:101F500090E00E940F066091920170919301809130
:101F60009401909195010C944706E82FF0E0E25E11
:101F7000FD4F80810895089580EA8A95F1F70895CC
:101F800000C008950C94BC0F08950C94C40F0C94D9
:101F9000C50F0C94C40F0C94C90FF894E82FE29568
:101FA000EF70F0E031A1282F2F7081E090E001C0A8
:101FB000880F2A95EAF7982F9095932391A392A1E1
:101FC000892B82A378940895CF93DF9385E30E94B1
:101FD000CD0F86E30E94CD0FCBE7D1E089918F3FF3
:101FE00011F00E94CD0F81E0C238D807B9F7DF9118
:101FF000CF910895CF92DF92EF92FF920F931F93AC
:10200000CF93DF938C01C62FD0E0CE018E579E4F29
:102010007C01FC0190819F3F09F447C0D62EF894C3
:10202000E92FE295EF70F0E081A19F7021E030E0B0
:1020300001C0220F9A95EAF7822B81A382A12095F5
:10204000282322A378940E94C00FEBE7F1E042E836
:1020500051E031E0C12C21912F3F89F0A22FA295B0
:10206000AF70B0E090968C9190E02F7002C0959583
:1020700087952A95E2F780FD02C0832F01C080E09A
:10208000C82A330F4E175F0731F7F70180818F3F62
:1020900011F00E94CD0F61E0C11001C060E08D2DF4
:1020A0000E94C20FC00FD11FC882DF91CF911F9134
:1020B0000F91FF90EF90DF90CF9008950E94E40F72
:1020C00010921F0210921E0210921D0210921C020A
:1020D00082E00E94A5100C9489011F93CF93DF9397
:1020E00000D0CDB7DEB71A82198260E0CE0101962A
:1020F0000E94FA0F61E0CE0101960E94FA0F42E0C1
:1021000050E0BE016F5F7F4F8CE192E00E94591E4C
:1021100011E0009709F410E0892B31F089819A8150
:1021200090931D0280931C02212F42E06EE172E029
:102130008CE192E00E94A6100E948B01812F0F90EB
:102140000F90DF91CF911F9108950895FF920F9303
:102150001F93CF93DF938C01F62ED72FC42F22230A
:1021600049F081E08093F3010E9401179093F201FE
:102170008093F1018091F3018823C1F08091F101F6
:102180009091F2010E941917059780F0EF2DFD2F15
:10219000D8014C2F50E0CD01801B910B841795077F
:1021A0001CF48D918193F7CF1092F301DF91CF91C1
:1021B0001F910F91FF9008950E94F1180E94DF0C6B
:1021C0000C94FD180E9401190E946D0D0C941B19AE
:1021D0000E949F160E94D8180E94CD0C0E94DC100D
:1021E0000E94E2100E94D70CFBCF8091FA0180FF81
:1021F00006C06091090170E0660F771F26C081FF5D
:1022000004C06091090184E005C082FF07C06091AD
:10221000090188E0689FB001112417C09091F9016D
:102220009923D1F060910801961788F72091090150
:1022300088E0289F90011124929FA001939F500D48
:10224000112470E0CA010E942B1E6038710540F411
:102250006115710519F406C068E070E0862F0895D5
:102260008FE7089581E008958091FA0180FF08C00A
:102270006091050170E0759567957595679521C02A
:1022800081FF06C06091050170E07595679519C0E2
:1022900082FF04C06091050170E010C09091F801C8
:1022A000992399F0609104019617A0F78091050198
:1022B000899FC001112470E00E942B1E60387105B7
:1022C00040F46115710519F406C061E070E0862FD5
:1022D00008958FE7089581E008958D3E21F40E94CE
:1022E000F510819504C08E3E29F40E94F51080936C
:1022F000FE0108958F3E21F40E94F510819504C0DF
:10230000803F29F40E94F5108093FD010895893FD4
:1023100019F40E94341105C08A3F31F40E9434112F
:1023200081958093FF0108958B3F21F40E94341121
:10233000819504C08C3F29F40E94341180930002DF
:1023400008959FE0980F983078F421E030E0A901DB
:1023500002C0440F551F9A95E2F7CA019091FC0103
:10236000892B8093FC0108958D3F21F48091FA011F
:1023700081600BC08E3F21F48091FA01826005C01C
:102380008F3F29F48091FA0184608093FA010895C7
:102390008D3E39F49091FE0197FF35C01092FE01F9
:1023A00059C08E3E29F49091FE011916BCF32BC042
:1023B0009091FD018F3E29F497FF25C01092FD01F9
:1023C00049C0803F19F41916CCF31DC09091FF014C
:1023D000893F29F41916BCF41092FF013BC08A3FD3
:1023E00019F497FF10C0F8CF8B3F39F49091000299
:1023F00097FF09C0109200022DC08C3F21F49091EC
:1024000000021916BCF39FE0980F983080F421E089
:1024100030E0A90102C0440F551F9A95E2F7CA01A6
:1024200080959091FC0189238093FC0113C08D3F1E
:1024300021F48091FA018E7F0BC08E3F21F48091B0
:10244000FA018D7F05C08F3F29F48091FA018B7FBF
:102450008093FA018091FD01811106C08091FE01F7
:10246000811102C01092F9018091FF01811106C013
:1024700080910002811102C01092F80108950E941B
:1024800001172091FD01211104C02091FE0122239A
:1024900021F09093F7018093F6012091FF01211123
:1024A00004C020910002222321F09093F501809333
:1024B000F4018BEF91E00C94DD15EF92FF920F93F6
:1024C0001F93CF93DF9300D000D000D0CDB7DEB7FD
:1024D00086E0EBEFF1E0DE01119601900D928A9516
:1024E000E1F7E090FD01F090FE010091FF011091F5
:1024F00000021092FD011092FE011092FF01109255
:102500000002E11003C0FF2009F45DC08091F601D4
:102510009091F7010E941917AC019091F90199234C
:1025200039F020910A0130E02417350758F04BC0EC
:1025300020910B018AE0289F900111242417350770
:1025400018F041C09F3F19F09F5F9093F901EE2072
:1025500061F00E94F5101E1414F09FEF01C091E08D
:10256000989F902D11249093FD01FF2061F00E940F
:10257000F5101F1414F09FEF01C091E0989F902D6B
:1025800011249093FE013091FD013323E1F020915D
:10259000FE012223C1F045EB3403C001112499232D
:1025A00019F09093FD0103C081E08093FD0135EBAC
:1025B0002303C0011124992319F09093FE0103C055
:1025C00081E08093FE01011103C0112309F45DC075
:1025D0008091F4019091F5010E941917AC0190913E
:1025E000F801992339F02091060130E024173507CE
:1025F00058F04BC0209107018AE0289F90011124D8
:102600002417350718F041C09F3F19F09F5F909342
:10261000F801002361F00E943411101614F09FEFAE
:1026200001C091E0989F902D11249093FF011123F8
:1026300061F00E943411111614F09FEF01C091E077
:10264000989F902D1124909300023091FF01332325
:10265000E1F0209100022223C1F045EB3403C001D8
:102660001124992319F09093FF0103C081E0809316
:10267000FF0135EB2303C0011124992319F0909336
:10268000000203C081E0809300028091FD0181116E
:102690000BC08091FE01811107C08091FF01811163
:1026A00003C08091000281110E943F12EB82FC82E4
:1026B0000D831E8386E0FE013196ABEFB1E0019001
:1026C0000D928A95E1F726960FB6F894DEBF0FBEFD
:1026D000CDBFDF91CF911F910F91FF90EF900895A3
:1026E000EBEFF1E086E0DF011D928A95E9F71092A9
:1026F000F9011092F8011092FA010895CF93DF9337
:10270000EC01FB018281882309F43CC1C430FDE562
:10271000DF0760F4CB3F9CE5D90788F49E01225087
:102720003C452431310508F02EC109C0C236EDE523
:10273000DE0729F0C63AFDE5DF0709F024C10E9453
:10274000060C90931B0280931A02C1318CE5D807C6
:1027500009F4C6C008F042C0C930ECE5DE0709F450
:102760009BC000F5C5308CE5D80709F485C078F426
:10277000C330ECE5DE0709F478C008F07AC0C23057
:10278000DC4509F0F5C080911A028160EFC0C730C6
:102790009CE5D90709F478C008F07AC080911A0244
:1027A0008061E4C0CD30FCE5DF0709F487C058F450
:1027B000CB309CE5D90709F479C008F07BC0809143
:1027C0001A0288606FC0CF30FCE5DF0709F480C0D3
:1027D00008F082C080911A02877FC8C0CE3F9CE576
:1027E000D90709F471C000F5C531FCE5DF0709F42C
:1027F00085C068F4C3319CE5D90709F475C008F0B9
:1028000095C00E94B70580911A028F77AFC0CC3F68
:10281000FCE5DF07A9F108F054C0CB3FDC4509F027
:10282000A7C080911B0240C0C230EDE5DE0709F46D
:1028300089C058F4C1158DE5D80709F45AC008F0CD
:1028400069C080911B0282602FC0C236EDE5DE07B1
:1028500009F47CC0C63AFDE5DF0709F481C0C33046
:10286000DD4509F085C080E06EC080911A0282606B
:102870007DC080911A0216C080911A02886076C0CD
:1028800080911B0282604FC080911A0280626EC0EC
:1028900080911A0280646AC00E94B70580911A0272
:1028A000806864C0846062C081603DC080911A020B
:1028B0008E7F5CC080911A028D7F58C080911A0271
:1028C00016C080911B0218C080911B028D7F2BC007
:1028D00080911A028F7E4AC080911A028F7D46C075
:1028E00080911A028F7B42C080911A02877F8B7F72
:1028F0003DC080911B028D7F8E7F15C080911A0292
:1029000082FB222720F991E0922790FB82F990FB2D
:1029100083F92CC080911B02982F909591708E7F27
:10292000892B90FB81F980931B0222C00E94B7057E
:1029300080911A0287FB222720F991E0922790FBD1
:1029400087F914C081E00E949D0C12C080911A0288
:1029500084FB222720F991E0922790FB84F906C09E
:1029600080911A02982F909590FB80F980931A021B
:1029700080911A0290911B020E94170C0E94B705C9
:1029800080E001C081E0DF91CF910895CF93DF9384
:1029900086319C4541F5EB010E940A0B982F8A81F4
:1029A0002091020130910301882379F09A7A81E025
:1029B00009F480E080930102911102C069E201C034
:1029C00065E3C9010E9459160AC080910102811174
:1029D00002C069E201C065E3C9010E945B160E9462
:1029E0004C0B80E001C081E0DF91CF9108950F93FF
:1029F0001F93CF93DF93C42FD22FFC0182818823B2
:102A0000C9F0409304020E9401179093030280933F
:102A1000020280E28C0F883008F057C0C77081E056
:102A200001C0880FCA95EAF7DF91CF911F910F91EE
:102A30000C94140380910402481330C08091020268
:102A4000909103020E941917883C910538F510E215
:102A50001D0FCD17B9F080E28C0F883040F4C7709D
:102A600081E001C0880FCA95EAF70E941B03183065
:102A700028F581E09D2F977001C0880F9A95EAF79D
:102A80000E941403802F0E940B031830F0F4D770BB
:102A900081E001C0880FDA95EAF70AC080E28C0F66
:102AA000883098F4C77081E001C0880FCA95EAF7B2
:102AB000DF91CF911F910F910C941B03802FDF9119
:102AC000CF911F910F910C940B03DF91CF911F9128
:102AD0000F9108950F939C01CB01243F4CE53407DF
:102AE00031F188F4293DFCE53F07D9F02A3D4CE55A
:102AF000340779F1283D3C45A9F506E221EE41EE87
:102B000068ED7CE52BC0263FFCE53F07E1F0A8F02F
:102B1000273F3C4539F507E225EE46EE67EF7CE5B9
:102B20001DC007E225EE45EE69ED7CE517C006E223
:102B300021EE40EE64EF7CE511C007E225EE44EEA5
:102B400065EF7CE50BC006E221EE42EE66EF7CE528
:102B500005C008E221E045EE6AED7CE50E94F7142D
:102B600080E008C0FC018281882319F010920402E1
:102B700001C081E00F9108959093850180938401B5
:102B8000089590930A02809309020895E091090242
:102B9000F0910A02309721F00190F081E02D099424
:102BA00080E00895E0910902F0910A02309721F047
:102BB0000280F381E02D09940895E0910902F091DB
:102BC0000A02309739F022E0DC012C930480F58171
:102BD000E02D0994089520910702309108022817EA
:102BE000390771F09093080280930702E09109027F
:102BF000F0910A02309721F00680F781E02D0994C8
:102C0000089520910502309106022817390771F0C6
:102C10009093060280930502E0910902F0910A0266
:102C2000309721F00084F185E02D09940895FC018E
:102C3000329697E080E0915029F021912223D9F338
:102C40008F5FF9CF0895662349F0FC01329608960C
:102C50002191621729F0E817F907D1F780E008956C
:102C600081E008959C01FC0132969FEF80E0419144
:102C7000461789F09F3F19F4411101C0982F8F5FCB
:102C80008630A9F79F3F39F0F901E90FF11D97FD53
:102C9000FA956283089508959C012A5F3F4FFC01D5
:102CA0004281461301C01282019682179307B9F739
:102CB00008950C9432160C944C16029626E0FC01F2
:102CC00011922A95E9F7089508950C94641683E00B
:102CD00080930B020C946516811102C081E001C043
:102CE00082E080930B020C9465160C946C1681E0C4
:102CF00080930B020C9465160C94771608950C942F
:102D00007E160C947F160C947E160C947E160C94F2
:102D10007E160E9485160E946D100E94831680E028
:102D20000E94B50F811108C081E00E94B50F91E0AB
:102D3000811103C090E001C091E0892F08950895AA
:102D40001F920F920FB60F9211248F939F93AF9300
:102D5000BF9380910C02811113C080912002909149
:102D60002102A0912202B09123024196A11DB11D22
:102D70008093200290932102A0932202B093230219
:102D8000BF91AF919F918F910F900FBE0F901F90A9
:102D9000189580912802843031F10E94EF01109241
:102DA0000C0220E488E190E00FB6F894A895809397
:102DB00060000FBE2093600083B7817F846083BF73
:102DC00083B7816083BF7894889583B78E7F83BFF4
:102DD0000FB6F894A8958091600088618093600098
:102DE000109260000FBE08950E94B7050C94F30185
:102DF00082E084BD93E095BD9AEF97BD80936E000D
:102E000008952FB7F8948091200290912102A0910B
:102E10002202B09123022FBF08952FB7F89460913A
:102E200020027091210280912202909123022FBFF3
:102E300008959C014FB7F89480912002909121024F
:102E4000A0912202B09123024FBF821B930B0895E1
:102E500078941F920F920FB60F9211248F939F9325
:102E6000AF93BF938091200290912102A091220202
:102E7000B09123020196A11DB11D80932002909371
:102E80002102A0932202B0932302BF91AF919F91A0
:102E90008F910F900FBE0F901F90189587E797E7BF
:102EA00090930108809300089AE088E10FB6F894A7
:102EB000A895809360000FBE90936000FFCF809133
:102EC00018020895089522E02093E9002FEF309131
:102ED000E800215035FD06C035ED3A95F1F70000C8
:102EE0002111F5CF2091E80025FF0BC040E050E014
:102EF00066E070E00E948D198091E8008E778093E3
:102F0000E8000895CF93DF9321E02093E9002FEFAD
:102F10003091E800215035FD06C035ED3A95F1F7C6
:102F200000002111F5CF2091E80025FF14C0EC012D
:102F300040E050E068E070E00E948D198091E80068
:102F40008E778093E80088E0FE01A0E1B2E0019076
:102F50000D928A95E1F7DF91CF91089580930D024C
:102F600070930F0260930E0280912802843001F565
:102F700082E08093E9008FEF9091E800815095FD09
:102F800006C095ED9A95F1F700008111F5CF80917B
:102F9000E80085FF0DC040E050E063E070E08DE0A8
:102FA00092E00E948D198091E8008E778093E8006E
:102FB0000895BC0184E00C94AE17BC0183E00C942E
:102FC000AE1780912702811109C00E941E1B0E942A
:102FD0007B1B8091E20084608093E2000895109250
:102FE000270208950C947C166091240281E06111FF
:102FF00001C080E00C9467169091280281E0943023
:1030000009F080E0609124020C946C1642E061ECBF
:1030100081E00E94971A42E261EC82E00E94971AD6
:103020009091280281E0943009F080E060912402C0
:103030000C94751680912A02833009F461C030F433
:10304000813071F0823009F49AC008958A3009F411
:1030500086C08B3009F46CC0893009F0A8C020C04C
:1030600080912902813A09F0A2C08091E800877F0F
:103070008093E80080912D0290912E02892B21F4FB
:1030800068E080E192E003C060E080E090E070E002
:103090000E94D8198091E8008B778093E80008950A
:1030A00080912902813209F082C080912D02909195
:1030B0002E02029708F07BC08091E800877F809302
:1030C000E8008091E80082FD05C08091280281110E
:1030D000F8CF6DC02091F3008091F20090E0922B28
:1030E000029731F48091F100813011F0863021F4A3
:1030F0008091F100809318028091E8008B7753C093
:1031000080912902813A09F052C080912D0290915C
:103110002E02892B09F04BC08091E800877F8093B5
:10312000E8008091E80080FFFCCF8091180136C054
:10313000809129028132D9F580912D0290912E0241
:10314000892BA9F58091E800877F8093E8000E9491
:10315000CC1A80912B02809318010C94B7058091B2
:103160002902813221F58091E800877F8093E80071
:103170000E94CC1A80912C028093190208958091AC
:103180002902813AA1F48091E800877F8093E800CA
:103190008091E80080FFFCCF809119028093F100BC
:1031A0008091E8008E778093E8000C94CC1A089503
:1031B00084B7877F84BF0FB6F894A895809160008C
:1031C000886180936000109260000FBE90E080E8FC
:1031D0000FB6F89480936100909361000FBE0C9439
:1031E00077160E941E1B0E947B1BE2EEF0E080819E
:1031F0008460808378940C94101E8CE091E00C9491
:10320000C115809128028530A9F48091280285306B
:1032100079F40E94C916809126028823B1F30E9496
:103220008916882391F30E9477190E94B705EDCF84
:103230000C94F416089508950C941E19292F332721
:1032400023303105C9F060F42130310581F022309E
:10325000310509F044C08BE390E028E231E043C03F
:1032600021323105E1F02232310549F138C082E1E5
:1032700090E023E631E037C099278130910549F08D
:1032800028F0029761F5E4EFF0E005C0E4E2F1E038
:1032900002C0E8E0F1E0849190E09F0124C0611554
:1032A000710541F061307105D1F489E090E023E5CA
:1032B00031E019C089E090E02AE331E014C06115E3
:1032C000710541F06130710551F48BE790E025E71D
:1032D00031E009C080E490E020EF31E004C080E0FC
:1032E00090E020E030E0FA0131832083089580E10E
:1032F00089BD82E189BD09B400FEFDCF8091D8006F
:103300008F7D8093D8008091E00082608093E00000
:103310008091E00081FDFCCF0895CF92DF92EF9283
:10332000FF920F931F93CF93DF93EC018B017A01F0
:103330000E94EB1A811133C0E114F10439F0F70156
:1033400080819181081B190BC80FD91FC12CD12C6A
:103350000115110519F18091E80085FD16C08091D5
:10336000E8008E778093E800E114F10449F0F7015A
:1033700080819181C80ED91ED182C08285E00FC0A4
:103380000E94EB1A882321F30AC089918093F100EF
:1033900001501109FFEFCF1ADF0ADACF80E0DF9189
:1033A000CF911F910F91FF90EF90DF90CF900895F4
:1033B00020912F02309130022617370748F061150F
:1033C000710539F42091E8002E772093E80001C0C0
:1033D000B901FC0120E06115710579F180912802A5
:1033E0008823F1F18530F1F18091E80083FD3CC044
:1033F0008091E80082FD2EC08091E80080FFEBCF35
:103400002091F3008091F20090E0922B61157105FC
:1034100051F08830910538F421912093F1006150EA
:1034200071090196F3CF21E0089709F020E080911F
:10343000E8008E778093E800CECF2111CFCF0AC06D
:1034400080912802882361F0853061F08091E80046
:1034500083FD0AC08091E80082FFF2CF80E00895EA
:1034600082E0089583E0089581E0089520912F027D
:10347000309130022617370748F06115710539F48D
:103480002091E8002E772093E80001C0B901FC01EB
:1034900020E06115710591F180912802882309F4DB
:1034A00040C0853009F43FC08091E80083FD3DC0F5
:1034B0008091E80082FD2FC08091E80080FFE9CF75
:1034C0002091F3008091F20090E0922B611571053C
:1034D00059F08830910540F424912093F100319601
:1034E000615071090196F2CF21E0089709F020E0C0
:1034F0008091E8008E778093E800CBCF2111CCCF6C
:103500000AC080912802882361F0853061F08091A3
:10351000E80083FD0AC08091E80082FFF2CF80E0DE
:10352000089582E0089583E0089581E00895982F3A
:10353000973068F59093E900981739F07091EC0096
:103540002091ED005091F00003C0242F762F50E021
:1035500021FD02C09F5FECCF3091EB003E7F3093A6
:10356000EB003091ED003D7F3093ED003091EB00AA
:1035700031603093EB007093EC002093ED0050939A
:10358000F0002091EE0027FDE5CF80E008958F70D8
:103590008093E90081E008958091290287FF11C09E
:1035A0008091E80082FD05C0809128028111F8CF4A
:1035B00011C08091E8008B770BC08091280288238E
:1035C00049F08091E80080FFF8CF8091E8008E7785
:1035D0008093E80008952091E4003091E50095E69D
:1035E0004091EC00842F817040FF23C08091E8005F
:1035F00080FD1DC080912802882399F0853099F0C4
:103600008091EB0085FD11C04091E4005091E500F0
:103610002417350729F3915011F09A01E1CF84E086
:10362000089582E0089583E0089581E0089580E0A0
:1036300008954091E80042FFDDCF08950E948C1B61
:103640000E94941BE0EEF0E0808181608083E8EDD1
:10365000F0E080818F77808319BCA7EDB0E08C917A
:103660008E7F8C9380818F7E8083109227020895B5
:103670000F931F93CF93DF930E948C1B0E94941B88
:10368000C8EDD0E088818F778883888180688883BF
:1036900088818F7D888319BC1092280210922402A1
:1036A000109226021092250200EE10E0F8018081AF
:1036B0008B7F808388818160888342E060E080E046
:1036C0000E94971AE1EEF0E080818E7F8083E2EE27
:1036D000F0E0808181608083808188608083F80150
:1036E00080818E7F8083888180618883DF91CF9104
:1036F0001F910F910895E8EDF0E080818F7E808327
:10370000E7EDF0E080818160808384E082BF81E02A
:10371000809327020C94381BE8EDF0E080818E7FC7
:1037200080831092E20008951092DA001092E10076
:1037300008951F920F920FB60F9211242F933F936B
:103740004F935F936F937F938F939F93AF93BF93A9
:10375000EF93FF938091E10082FF0BC08091E20024
:1037600082FF07C08091E1008B7F8093E1000E947F
:103770000F1E8091DA0080FF1FC08091D80080FF6B
:103780001BC08091DA008E7F8093DA008091D9008F
:1037900080FF0DC080E189BD82E189BD09B400FED2
:1037A000FDCF81E0809328020E94E11705C019BC7B
:1037B000109228020E94EF178091E10080FF19C04B
:1037C0008091E20080FF15C08091E2008E7F80939F
:1037D000E2008091E20080618093E2008091D80055
:1037E00080628093D80019BC85E0809328020E94F3
:1037F000F4178091E10084FF30C08091E20084FFE3
:103800002CC080E189BD82E189BD09B400FEFDCFF5
:103810008091D8008F7D8093D8008091E1008F7EC9
:103820008093E1008091E2008F7E8093E20080919E
:10383000E20081608093E20080912402882311F0ED
:1038400084E007C08091E30087FD02C081E001C0F1
:1038500083E0809328020E94FC178091E10083FF9F
:1038600029C08091E20083FF25C08091E100877F1D
:103870008093E10082E080932802109224028091DC
:10388000E1008E7F8093E1008091E2008E7F809343
:10389000E2008091E20080618093E20042E060E01B
:1038A00080E00E94971A8091F00088608093F00079
:1038B0000E94F217FF91EF91BF91AF919F918F916D
:1038C0007F916F915F914F913F912F910F900FBE1C
:1038D0000F901F9018951F920F920FB60F92112400
:1038E0002F933F934F935F936F937F938F939F9308
:1038F000AF93BF93CF93DF93EF93FF93C091E90012
:10390000CF708091EC00D82FD17080FDD0E810925C
:10391000E9008091F000877F8093F00078940E9406
:10392000AF1C1092E9008091F00088608093F00055
:10393000CD2BCF70C093E900FF91EF91DF91CF9134
:10394000BF91AF919F918F917F916F915F914F91B7
:103950003F912F910F900FBE0F901F9018951F93BE
:10396000CF93DF93CDB7DEB7AA970FB6F894DEBF3B
:103970000FBECDBFE9E2F2E08091F100819322E039
:10398000E133F207C9F70E941A188091E80083FF1B
:103990002EC18091290290912A02492F50E04A308D
:1039A000510508F024C1FA01EE59FF4F0C943F1E57
:1039B000803821F0823809F01AC108C080912502B0
:1039C00090912602992389F082600FC080912D0288
:1039D0008F70873008F00BC18093E9008091EB0075
:1039E00085FB882780F91092E9009091E800977F85
:1039F0009093E8008093F1001092F100D1C0282F3D
:103A00002D7F09F0F4C0882319F0823061F0EFC0F7
:103A100080912B02813009F0EAC0933009F080E0F8
:103A2000809326022EC080912B0281112AC08091A2
:103A30002D028F702FEF280F263008F0D8C080930A
:103A4000E9002091EB0020FF1CC0933021F480910D
:103A5000EB00806214C09091EB0090619093EB00BA
:103A600021E030E0A90102C0440F551F8A95E2F71A
:103A70004093EA001092EA008091EB008860809306
:103A8000EB001092E9008091E800877F8093E800C6
:103A90000E94CC1AACC08111AAC010912B021F77D2
:103AA0008091E3008078812B8093E3008091E8008F
:103AB000877F8093E8000E94CC1A8091E80080FF05
:103AC000FCCF8091E30080688093E300111102C075
:103AD00082E001C083E08093280289C08058823050
:103AE00008F085C080912B0290912C028C3D53E010
:103AF000950779F583E08A838AE289834FB7F89442
:103B0000DE01139620E03EE051E2E32FF0E0509317
:103B10005700E49120FF03C0E295EF703F5FEF7024
:103B20008E2F90E0EA3010F0C79601C0C0968D93BA
:103B30009D932F5F243149F74FBF8091E800877F25
:103B40008093E8006AE270E0CE0101960E94D819E5
:103B500016C060912D0270912E02AE014F5F5F4F33
:103B60000E941C19BC01892B09F441C09091E80006
:103B7000977F9093E80089819A810E94361A8091FC
:103B8000E8008B778093E80032C0803881F580911F
:103B9000E800877F8093E800809124028093F10001
:103BA0008091E8008E7772CF811121C080912B0225
:103BB00090912C0299270297D4F48091E800877F96
:103BC0008093E80080912B02809324020E94CC1AFB
:103BD00080912402811106C08091E30087FD02C01C
:103BE00081E001C084E0809328020E940618809141
:103BF000E80083FF0AC08091E800877F8093E80097
:103C00008091EB0080628093EB00AA960FB6F89447
:103C1000DEBF0FBECDBFDF91CF911F9108950895F4
:103C2000CF93809128028823A1F0C091E900CF7042
:103C30009091EC00892F817090FD80E8C82B109244
:103C4000E9008091E80083FD0E94AF1CCF70C09313
:103C5000E900CF91089597FB072E16F4009407D042
:103C600077FD09D00E94451E07FC05D03EF49095D3
:103C700081959F4F0895709561957F4F0895EE0F40
:103C8000FF1F0590F491E02D0994AA1BBB1B51E185
:103C900007C0AA1FBB1FA617B70710F0A61BB70BBC
:103CA000881F991F5A95A9F780959095BC01CD0161
:103CB0000895FB01DC0104C08D910190801921F46D
:103CC00041505040C8F7881B990B0895F999FECFD1
:103CD00092BD81BDF89A992780B50895A8E1B0E01A
:103CE00042E050E00C949A1E262FF999FECF92BD27
:103CF00081BDF89A019700B4021639F01FBA20BDB1
:103D00000FB6F894FA9AF99A0FBE08950396272FE2
:103D10000E94751E0E94741E252F0E94751E242F5E
:103D20000C94751E0196272F0E94751E0C94741E0C
:103D3000DC01CB01FC01F999FECF06C0F2BDE1BD6B
:103D4000F89A319600B40D9241505040B8F708955A
:043D5000F894FFCF15
:103D5400C800DC01280850011E0A14015F178217ED
:103D64006317DD17D917621701E200E900EA00B50D
:103D740000B600B700CD008301CC008A0192019403
:103D8400012102230224022502260227022A02B369
:103D940000B4006F007000818283E200E900EA0051
:103DA400B500B600B700CD008301CC008A019201B2
:103DB40094012102230224022502260227022A0258
:103DC400B300B4006F00700081828397C63432332D
:043DD40031F7353658
:00000001FF
